:100000009EC09DC544C59BC59AC599C598C597C551
:1000100096C595C594C593C592C591C590C58FC524
:100020008EC58DC58CC58BC58AC589C588C587C554
:1000300086C585C584C583C582C581C580C53E008A
:100040003E0A800000407A10F35A00A0724E180950
:100050000010A5D4E80000E87648170000E40B542F
:10006000020000CA9A3B000000E1F50500008096FE
:100070009800000040420F000000A0860100000030
:10008000102700000000E8030000000064000000EA
:1000900000000A00000000000100000000002C76B3
:1000A000D888DC674F0823DFC1DFAE59E1B1B796CE
:1000B000E5E3E453C63AE651997696E8E6C284262B
:1000C000EB898C9B62ED407C6FFCEFBC9C9F40F207
:1000D000BAA56FA5F490055A2AF75C936B6CF96783
:1000E0006DC11BFCE0E40D47FEF520E6B500D0ED48
:1000F000902E0300943577050080841E08000020B0
:100100004E0A000000C80C333333330F986E12834D
:100110001141EF8D2114893BE65516CFFEE6DB1821
:10012000D1844B381BF77C1D901DA4BBE4242032E6
:1001300084725E228100C9F124ECA1E53D271124DF
:100140001FBECFEFCDBFDFE3DEBFEEE3F0E040E068
:1001500017C0B591A59135912591059107FD0CC06A
:1001600095918591EF01F92FE82F05900D92A21737
:10017000B307D9F7FE0104C01D92A217B307E1F738
:0E018000E334F40731F75BD300C0F894FFCFEF
:10018E0053696E676C652053616D706C65643A20BF
:10019E0000560D0A004F7665722053616D706C65C6
:0A01AE00643A2000560D0A0D0A0005
:1001B800A9E0B0E0E1EEF0E018C46A01122FB02E19
:1001C8002BE3201720F0FF24F394F00E02C02CE359
:1001D800F22E0F2D27E0AE014F5F5F4F40D1BC01DB
:1001E8004981842F8970813031F0E1FC06C0E0FE3E
:1001F80006C090E205C09DE203C09BE201C090E00A
:100208005E2D507143FF3CC0911102C083E001C0D4
:1002180084E0811718F4212F281B01C020E0511118
:100228000BC0F601822F30E2882319F031938150F8
:10023800FBCFC20ED11C20E0992329F0D6019C9354
:10024800F60131966F01C6010396E2FE0AC03EE44C
:10025800D6013C9341E411964C93119712963C9326
:1002680006C03EE6F601308341E641833283FC0155
:10027800322F40E2332309F442C041933150FACF80
:1002880042FF44C0911102C083E001C084E081179D
:1002980018F4212F281B01C020E051110BC0F601D2
:1002A800822F30E2882319F031938150FBCFC20EA0
:1002B800D11C20E0992329F0D6019C93F6013196B0
:1002C8006F01C6010396E2FE0BC039E4D6013C93E8
:1002D8003EE411963C93119736E412963C9307C07E
:1002E80039E6F60130833EE6318336E63283FC0197
:1002F800322F40E2332319F041933150FBCFFC01F8
:10030800E20FF11D10828EEF9FEFA6C021E030E0D2
:10031800911102C020E030E0161617061CF4FB010C
:10032800319602C0E1E0F0E02E0F3F1FBB2021F024
:10033800EB2DF0E0319602C0E0E0F0E02E0F3F1F19
:10034800E12FF0E02E173F071CF4121B212F01C0EC
:1003580020E08E2D887159F4F601822F30E288232F
:1003680019F031938150FBCFC20ED11C20E09923A4
:1003780029F0D6019C93F60131966F0151110BC0FB
:10038800F601822F90E3882319F091938150FBCFD7
:10039800C20ED11C20E00F2D060F9A81342F307128
:1003A80044FF03C0913309F40150101624F40930B6
:1003B80018F008E001C001E0AB0177FF02C040E09F
:1003C80050E0FB01E41BF50BA1E0B0E0AC0FBD1F52
:1003D800EA0FFB1F8EE2A82E4B01801A91080B2D05
:1003E80010E01195019511094F3FBFEF5B0721F40C
:1003F800D601AC9211966D01641775072CF084161E
:10040800950614F4818101C080E341505109319669
:10041800D60111967D014017510724F0D6018C931F
:100428006701E2CF6417750739F4963320F49533E2
:1004380019F4311101C081E3F6018083F701822F9D
:1004480090E2882319F091938150FBCFF701E20FD6
:0E045800F11D108280E090E02996ECE0DFC2FA
:10046600283008F027E03327DA01990F311D87FD80
:10047600916000966105710539F432602E5F3D93F7
:1004860030E32A95E1F708959F3F30F080387105F3
:10049600610509F03C5F3C5F3D93913008F0806850
:1004A600911DDF93CF931F930F93FF92EF92192F16
:1004B600987F9695E92F96959695E90FFF27E25630
:1004C600FF4F99273327EE24FF24A701E701059064
:1004D6000894079428F4360FE71EF81E491F511D8D
:1004E600660F771F881F991F0694A1F7059007943A
:1004F60028F4E70EF81E491F561FC11D770F881FE7
:10050600991F661F0694A1F70590079428F4F80E24
:10051600491F561FC71FD11D880F991F661F771FBA
:100526000694A1F70590079420F4490F561FC71F9C
:10053600D81F990F661F771F881F0694A9F7849105
:100546001095177041F0D695C79557954795F7942E
:10055600E7941A95C1F7E4E4F0E0689415901591D4
:1005660035916591959105907FE27395E118F10AB1
:10057600430B560BC90BD009C0F7E10CF11E431F04
:10058600561FC91FD01D7EF4703311F48A95E6CF2D
:10059600E894015030F0080F0AF40027021708F417
:1005A600202F2395022F7A3328F079E37D932A951D
:1005B600E9F710C07D932A9589F606949795679575
:1005C600379517951794E118F10A430B560BC90B8B
:1005D600D00998F023957E9173957A3308F070E3ED
:1005E6007C932013B8F77E9170617D9330F08395EC
:1005F60071E37D9370E32A95E1F71124EF90FF9064
:100606000F911F91CF91DF91992787FD90950895BE
:100616000E947A0558F00E94730540F029F45F3F66
:1006260029F00C948E0551110C9482050C949C05AE
:100636000E94790468F39923B1F3552391F3951B2E
:10064600550BBB27AA2762177307840738F09F5FED
:100656005F4F220F331F441FAA1FA9F335D00E2E5A
:100666003AF0E0E832D091505040E695001CCAF7C7
:100676002BD0FE2F29D0660F771F881FBB1F26178A
:1006860037074807AB07B0E809F0BB0B802DBF0161
:10069600FF2793585F4F3AF09E3F510578F00C9430
:1006A6008E050C9482055F3FE4F3983ED4F386955D
:1006B60077956795B795F7959F5FC9F7880F911D51
:1006C6009695879597F90895E1E0660F771F881F3D
:1006D600BB1F621773078407BA0720F0621B730BF0
:0C06E600840BBA0BEE1F88F7E095089516
:1006F2000E94730538F00E947A0520F0952311F0CC
:100702000C948E050C949C0511240C9482050E9475
:10071200790470F3959FC1F3950F50E0551F629FC6
:10072200F001729FBB27F00DB11D639FAA27F00D48
:10073200B11DAA1F649F6627B00DA11D661F829F6F
:100742002227B00DA11D621F739FB00DA11D621F54
:10075200839FA00D611D221F749F3327A00D611D71
:10076200231F849F600D211D822F762F6A2F112453
:100772009F5750409AF0F1F088234AF0EE0FFF1F86
:10078200BB1F661F771F881F91505040A9F79E3FDD
:10079200510580F00C948E050C9482055F3FE4F3C2
:1007A200983ED4F3869577956795B795F795E79533
:1007B2009F5FC1F7FE2B880F911D9695879597F93C
:0207C200089598
:1007C400E89409C097FB3EF49095809570956195E7
:1007D4007F4F8F4F9F4F9923A9F0F92F96E9BB279D
:1007E4009395F695879577956795B795F111F8CF19
:1007F400FAF4BB0F11F460FF1BC06F5F7F4F8F4F84
:100804009F4F16C0882311F096E911C0772321F079
:100814009EE8872F762F05C0662371F096E8862F11
:1008240070E060E02AF09A95660F771F881FDAF768
:0A083400880F9695879597F90895AF
:10083E0010920004E0E2F4E08FEF848384E0808382
:10084E0044D15FD139D129D06FD08EE891E827D12C
:10085E006091063E7091073E8091083E9091093E50
:10086E00A2D08FE991E81BD183EA91E818D160916B
:10087E00003E7091013E8091023E9091033E93D0D6
:10088E0082EB91E80CD12FEF88E09DE32150804060
:0A089E009040E1F700C00000D6CF43
:1008A80084E08093010685E090E0CAD0969587950C
:1008B800969587958093043E9093053EBC0180E011
:1008C80090E07CDF20E030E040E250E42DD120E0F1
:1008D80030EF4FE755E424D16093003E7093013E1A
:0A08E8008093023E9093033E0895B2
:1008F20057FD9058440F551F59F05F3F71F04795CF
:10090200880F97FB991F61F09F3F79F087950895B3
:10091200121613061406551FF2CF4695F1DF08C0D2
:10092200161617061806991FF1CF869571056105EF
:040932000894089588
:100936001092010685E090E084D08093043E909367
:10094600053EBC0180E090E03ADF20E030E040E286
:1009560050E4EBD020E030EC4FE754E4E2D0609373
:10096600063E7093073E8093083E9093093E089595
:10097600EF920F931F93CF93DF93E80147FD02C0D9
:1009860034E001C034E1042E000C550B57FF03C0C0
:10099600519541955109E32E022F242FAE0109DC12
:0E09A600CE01DF91CF911F910F91EF90089538
:1009B4000F931F93CF93DF93CDB7DEB7E297CDBFED
:1009C400DEBF8E010F5F1F4F24E041E0D2DFC8017C
:1009D4006BD0E296CDBFDEBFDF91CF911F910F9117
:0209E400089574
:1009E6002F923F924F925F926F927F928F929F9239
:1009F600AF92BF92CF92DF92EF92FF920F931F9327
:100A0600CF93DF93CDB7DEB7CA1BDB0BCDBFDEBFFF
:020A1600099441
:100A18002A88398848885F846E847D848C849B8486
:100A2800AA84B984C884DF80EE80FD800C811B8194
:100A3800AA81B981CE0FD11DCDBFDEBFED010895CA
:100A4800E0E0F6E0868381E0808780910B0680FFF6
:100A5800FCCFE0E0F6E020893189938591609387A7
:040A6800C901089523
:100A6C00092E0394000C11F4882352F0BB0F40F4B0
:100A7C00BF2B11F460FF04C06F5F7F4F8F4F9F4FF0
:020A8C000895CB
:100A8E001F920F920FB60F9211248F9381E08093D5
:0E0A9E008A008F910F900FBE0F901F90189539
:100AAC00FC0107C09091040895FFFCCF80930208CD
:0A0ABC00319680818111F6CF089574
:100AC600E0E0F8E08DE695E08087918780E4868314
:020AD600089581
:0E0AD80080E28093A00082E08093A100089548
:0E0AE60000240A94161617061806090608952D
:0E0AF40000240A94121613061406050608952F
:0E0B0200E894BB2766277727CB0197F9089563
:0C0B1000E0E0F6E081E08283808308953D
:0C0B1C0097F99F6780E870E060E00895A2
:080B28000E941B030C9436052A
:080B30000E9488030C943605B5
:060B38009FEF80EC089520
:020B3E0060CA8B
:02000004008278
:090000000000020000C40700002A
:00000001FF
